:020000040000FA
:040000001C20462852
:040004000034003490
:08000800F300030EF400831263
:10001000031383130408F5000A08F6008A018C18FC
:1000200055208C1ADD2176088A0075088400740E2C
:100030008300F30E730E0900830103018500F100B4
:100040008600F2008316E0308500073086008312B8
:1000500083161630810083120C3097000030950013
:100060008316FF30920083120430920007309F0005
:10007000243083169800903083129800273083161E
:1000800099008C16831281018B010800F023042152
:10009000532083168C1483120B178B17112403180B
:0600A0004E280B214E2842
:0A00A600F70108008C107708803E77
:1000B0009500F7018316031320102408A1072508D3
:1000C0000318250FA20726080318260FA307A01C54
:1000D0006F28230883169B001C141A08F707831641
:1000E00003132D103108AE0732080318320FAF0783
:1000F00033080318330FB007AD1C8428300883166B
:100100009B001C141A08F707831603133A103E08C5
:10011000BB073F0803183F0FBC0740080318400FF8
:10012000BD07BA1C99283D0883169B001C141A08A9
:10013000F7078316031347104B08C8074C0803182A
:100140004C0FC9074D0803184D0FCA07C71CAE282E
:100150004A0883169B001C141A08F707831603131A
:1001600054105808D50759080318590FD6075A08CC
:1001700003185A0FD707D41CC328570883169B00AF
:100180001C141A08F7078312031331103508B2073D
:1001900036080318360FB30737080318370FB407AC
:1001A000B11CD828340883169B001C141A08F707C2
:1001B000831203133E104208BF0743080318430F7E
:1001C000C00744080318440FC107BE1CED284108AE
:1001D00083169B001C141A08F707831203134B1095
:1001E0004F08CC0750080318500FCD0751080318CB
:1001F000510FCE07CB1C02294E0883169B001C14FE
:080200001A08F7078312080039
:080208000301061C0830D900B7
:10021000DE015A102D29DB00DB1F1A29F8305B02A2
:10022000031808005A105B08DE00F0305B02031868
:10023000DE0108005A1C1F29E0005A107429DE084C
:1002400003190800DF00C0305E02031C2B29E030D8
:100250005E02031C74295A140800A030A900AD30B6
:10026000AA00BA30AB00C730AC00D430AD0031309A
:10027000AE003E30AF004B30B000DB0129305B07F1
:1002800084000008E1006108003E840080016108EC
:10029000013E84008001840A8001840A8001610893
:1002A000043E84008001840A8001840A8001610880
:1002B000073E84003C3080006108083E84008001D5
:1002C000840A800161080A3E8400023080006108CF
:1002D0000B3E84007F308000840A8000DB0A0830F7
:1002E0005B02031D3E2908000F305E05E10059083E
:1002F000E102031C080008306102031808006108CD
:10030000293E84000008E10002308A005E0E0739B1
:10031000F03E820002308A005F08003E8200E00862
:06032000031DF82A052B65
:0A0326002008FC39A5002108A600FC
:10033000A7010C30A602031C9F29A70A9A29A60729
:100340000310A60CA50C0310260CA800250CA5076D
:1003500028080318280FA6070030A5070318A60AC7
:100360000730A607D9218A01A200A50A0319A60A07
:10037000D9218A01A300A50A0319A60AD9218A0155
:10038000A400A70E270E0A3C031C0301A700A71D0B
:10039000CF292308A2002408A300A401A711A708BD
:1003A0000319D8290310A40CA30CA20CA70BD22963
:0A03B000080026088A0025088200D4
:0603BA0070101819E4297F
:1003C0009818E7291A08F92B1A087014EA29181244
:0603D0001816701408006D
:10040000080008000800080008000800802A08000A
:10041000080008000800080008000800080008009C
:10042000080008000800080008000800080008008C
:10043000080008000800080008000800080008007C
:10044000080008000800080008000800080008006C
:10045000080008000800080008000800080008005C
:10046000080008000800080008000800080008004C
:10047000080008000800080008000800080008003C
:10048000080008000800080008000800080008002C
:10049000080008000800080008000800080008001C
:1004A000080008000800080008000800080008000C
:1004B00008000800080008000800080008000800FC
:1004C000922AA22AB12AB12AB92ABF2A0800080012
:1004D00008000800080008000800080008000800DC
:1004E00008000800080008000800080008000800CC
:1004F000182B312B182B182B182B182B182B182BCB
:1005000061080B3E84000008840A0004031D0800F3
:100510000D3060020318080061080A3E840060087C
:100520008000080061080B3E84000008840A000473
:10053000031D080061080A3E84000C300002031D00
:10054000800A080061080B3E84000008840A000449
:10055000031D080061080A3E84000008031D800393
:10056000080061080B3E84007F308000840A800010
:10057000080061080B3E84006008800008006108E4
:0A0580000C3E8400600880000800B3
:1005E000052B8F2908008A2908000800492B0800DC
:1005F0006108073E84005F08800092236108003E86
:100600008400801400148B1708006108073E8400E2
:100610005F080002031D08006108003E8400801C82
:1006200008000018112B8B13801000148B17080082
:1006300061080A3E840002308000013084077F3068
:100640008000840A80006108083E84008001840ADA
:10065000800192236108003E8400801000148B17F3
:10066000080061080A3E84000230800001308407DF
:100670007F308000840A80006108083E8400800189
:10068000840A800192236108003E840000148B17C5
:10069000080061080A3E840000085D236108083EE6
:1006A000840064088000840A650880009223610841
:1006B000003E840000148B170800E401E501DB0014
:1006C0005B080319912B0310DB0D0310DF0D0310E2
:1006D000DF0DE00D8030E0076008DC00DC1F782BC8
:1006E0005F08DF01DF026008E001031C013EE00259
:1006F0000830DD00DB0C031C832B5F08E407600877
:100700000318600FE507E50CE40CDD0B7A2BDC1F0A
:10071000912B6408E401E4026508E501031C013E35
:10072000E50208006108073E84000008A1000230CD
:1007300084070008A107A11FA42B0C30801FA22B47
:10074000A1029B2BA1079B2B84030008A0009321EF
:100750006108003E84000018AB2B6108043E840051
:100760008B1322088000840A23088000840A24084E
:0407700080000800FD
:1007E00003178317E0012030E200E10003138313B5
:1007F000080003178317E300601B0D2C62088400B8
:1008000063088000E00AE20A60306202031D0A2CDD
:100810002030E200031383130800031383137014C2
:10082000080003178317E0080319272C61088400C8
:100830000008E400E003E10A60306102031D222C9D
:100840002030E1006408031383130310080003132E
:06085000831303140800ED
:100E0000D434BB346D343234D5346D349534EE344F
:100E10006D34FE3407346E346E3421346E34E33472
:100E20003A346E345D3454346E34DE346D346E34A2
:100E3000653487346E34F134A0346E348434BA347B
:100E40006E341C34D4346E34BB34ED346E345F34C1
:100E500007346F34093421346F34B9343A346F3481
:100E60006F3454346F342B346E346F34ED34873434
:100E70006F34B534A1346F348334BB346F3457349A
:100E8000D5346F343034EF346F3410340934703467
:100E9000F63422347034E2343C347034D334563473
:100EA0007034CB3470347034C9348A347034CC34F8
:100EB000A4347034D634BE347034E634D83470344C
:100EC000FC34F234703417340D347134393427342F
:100ED00071346134413471348F345B347134C334D0
:100EE00075347134FD348F3471343D34AA34713427
:100EF0008334C4347134CF34DE3471342234F93461
:100F000071347A3413347234D9342D3472343D341C
:100F100048347234A8346234723419347D347234F3
:100F20009034973472340D34B23472349034CC34FB
:100F300072341934E7347234A834013473343E34D3
:100F40001C347334DA34363473347B3451347334B0
:100F500023346C347334D234863473348634A134FD
:100F600073344034BC3473340134D7347334C834EC
:100F7000F134733495340C34743468342734743455
:100F800042344234743421345D3474340734783458
:100F90007434F33492347434E634AD347434DE345F
:100FA000C8347434DD34E3347434E234FE347434DD
:100FB000ED3419347534FF34343475341634503408
:100FC000753434346B347534593486347534833421
:100FD000A1347534B434BC347534EB34D73475343F
:100FE0002934F33475346C340E347634B634293401
:100FF00076340734453476345D3460347634BA342C
:101000007B3476341D34973476348734B234763476
:10101000F734CD3476346D34E9347634EA3404343C
:1010200077346D3420347734F6343B347734863477
:10103000573477341C3473347734B9348E3477347E
:101040005B34AA3477340534C6347734B434E134AD
:1010500077346A34FD347734273419347834EA34F9
:1010600034347834B3345034783483346C34783452
:101070005934883478343534A43478341834C0344E
:1010800078340234DC347834F234F7347834E834A9
:1010900013347934E5342F347934E8344B347934EB
:1010A000F234673479340234843479341934A03416
:1010B00079343634BC3479345A34D834793484347D
:1010C000F4347934B53410347A34EC342C347A3442
:1010D0002A3449347A346E3465347A34B9348134FC
:1010E0007A340A349E347A346234BA347A34C0346E
:1010F000D6347A342534F3347A3491340F347B3453
:1011000003342C347B347C3448347B34FB346434F7
:101110007B34813481347B340E349E347B34A1346F
:10112000BA347B343A34D7347B34DB34F3347B3415
:10113000823410347C342F342D347C34E3344934FD
:101140007C349E3466347C34603483347C3428347C
:10115000A0347C34F634BC347C34CC34D9347C3484
:10116000A834F6347C348B3413347D347434303406
:101170007D3464344D347D345B346A347D34593489
:1011800087347D345D34A4347D346834C1347D3497
:101190007934DE347D349234FB347D34B134183408
:1011A0007E34D63435347E34033453347E3436348E
:1011B00070347E3470348D347E34B134AA347E344D
:1011C000F934C7347E344734E5347E349C340234F9
:1011D0007F34F8341F347F345A343D347F34C43480
:1011E0005A347F34343478347F34AB3495347F349C
:1011F0002934B3347F34AE34D0347F343934EE34D0
:101200007F34CC340B348034653429348034053455
:1012100047348034AC34643480345934823480347C
:101220000E34A0348034C934BD3480348C34DB3483
:1012300080345534F9348034253417348134FC3407
:1012400034348134DA3452348134BE3470348134ED
:10125000AA348E3481349D34AC3481349634CA340B
:1012600081349734E83481349E3406348234AC348B
:1012700024348234C23442348234DE3460348234E2
:1012800001347F3482342B349D3482345C34BB345B
:1012900082349434D9348234D334F73482341934D8
:1012A00016348334663434348334BB345234833458
:1012B00016347134833478348F348334E134AD346C
:1012C00083345134CC348334C834EA3483344634E0
:1012D00009348434CC342734843458344634843448
:1012E000EB34643484348634833484342734A23435
:1012F0008434D034C03484348034DF34843437349C
:10130000FE348434F4341C348534B9343B348534AD
:1013100086345A34853459347934853433349834A6
:1013200085341534B7348534FD34D5348534ED3403
:10133000F4348534E43413348634E234323486347D
:10134000E73451348634F4347034863407349034BE
:1013500086342234AF3486344434CE3486346D340B
:10136000ED3486349E340C348734D5342B348734B2
:1013700014344B3487345A346A348734A73489346C
:101380008734FC34A83487345734C8348734BA34AB
:10139000E734873425340734883496342634883447
:1013A0000F34463488348F346534883416348534A9
:1013B0008834A534A43488343B34C4348834D834D5
:1013C000E33488347C340334893428342334893436
:1013D000DB3442348934963462348934583482346C
:1013E00089342134A2348934F134C1348934C93484
:1013F000E1348934A83401348A348F3421348A3476
:101400007D3441348A34723461348A346F348134A7
:101410008A347334A1348A347E34C1348A349134AA
:10142000E1348A34AC3401348B34CD3421348B3400
:10143000F73441348B34273462348B345F34823454
:101440008B349F34A2348B34E634C2348B3434343E
:10145000E3348B348A3403348C34E73423348C34CF
:101460004C3444348C34B93464348C342C34853466
:101470008C34A834A5348C342A34C6348C34B53436
:10148000E6348C34473407348D34E03427348D34DB
:10149000813448348D34293469348D34DA348934D4
:1014A0008D349134AA348D345034CB348D34173488
:1014B000EC348D34E5340C348E34BB342D348E341E
:1014C00099344E348E347E346F348E346A34903492
:1014D0008E345F34B1348E345A34D2348E345E3428
:1014E000F3348E34693414348F347C3435348F348F
:1014F000963456348F34B83477348F34E234983499
:101500008F341334BA348F344D34DB348F348D340C
:10151000FC348F34D6341D34903426343F34903428
:101520007E3460349034DD34813490344534A334D7
:101530009034B434C43490342A34E6349034A9342A
:10154000073491342F3429349134BD344A349134E2
:1015500052346C349134F0348D3491349534AF344A
:1015600091344234D1349134F734F2349134B33479
:1015700014349234783436349234443458349234B7
:1015800018347A349234F4349B349234D734BD34E2
:101590009234C334DF349234B63401349334B134EA
:1015A00023349334B43445349334BF3467349334A0
:1015B000D23489349334ED34AB3493340F34CE3495
:1015C00093343A34F03493346C3412349434A63473
:1015D00034349434E8345634943432347934943492
:1015E00084349B349434DE34BD3494344034E03459
:1015F0009434AA34023495341B342534953495340C
:101600004734953417346A349534A0348C34953487
:101610003234AF349534CC34D13495346D34F43421
:101620009534173417349634C834393496348234A8
:101630005C34963444347F3496340D34A23496347A
:10164000DF34C4349634B934E73496349B340A34E6
:10165000973485342D34973477345034973471343B
:10166000733497347334963497347D34B934973463
:101670009034DC349734AA34FF349734CD34223498
:101680009834F734453498342A34693498346534BE
:101690008C349834A834AF349834F334D23498343A
:1016A0004734F6349834A2341934993406343D342E
:1016B0009934723460349934E63483349934623422
:1016C000A7349934E734CA3499347434EE349934F5
:1016D000093412349A34A63435349A344B3459349C
:1016E0009A34F9347C349A34AF34A0349A346D345B
:1016F000C4349A343334E8349A3402340C349B348E
:10170000D9342F349B34B83453349B349F347734DA
:101710009B348F349B349B348734BF349B34883460
:10172000E3349B34913407349C34A2342B349C34FE
:10173000BB344F349C34DD3473349C3407349834D8
:101740009C343A34BC349C347434E0349C34B83423
:1017500004349D34033429349D3457344D349D343E
:10176000B43471349D34183496349D348634BA348C
:101770009D34FB34DE349D34793403349E3400349C
:1017800028349E348F344C349E34263471349E3445
:10179000C63495349E346E34BA349E341F34DF34EC
:1017A0009E34D83403349F349A3428349F346434BC
:1017B0004D349F34373472349F34123497349F340D
:1017C000F634BB349F34E234E0349F34D7340534EC
:1017D000A034D5342A34A034DB344F34A034E93477
:1017E0007434A03400349A34A0342034BF34A0348C
:1017F0004834E434A03479340934A134B2342E347A
:10180000A134F4345334A1343F347934A1349234C4
:101810009E34A134EE34C334A1345334E934A134BA
:10182000C0340E34A23435343434A234B434593490
:10183000A2343B347F34A234CB34A434A234633496
:10184000CA34A2340534F034A234AE341534A3348F
:1018500061343B34A3341C346134A334E034863423
:10186000A334AD34AC34A3348334D234A3346134E0
:10187000F834A33448341E34A43437344434A43404
:1018800030346A34A43431349034A4343B34B63424
:10189000A4344E34DC34A4346A340234A5348E3497
:1018A0002834A534BC344E34A534F2347434A53411
:1018B00031349B34A5347934C134A534C934E73488
:1018C000A53423340E34A63485343434A634F034AD
:1018D0005A34A63464348134A634E134A734A634AF
:1018E0006734CE34A634F634F434A6348E341B3444
:1018F000A7342E344234A734D8346834A7348A3419
:101900008F34A7344634B634A7340A34DD34A734D0
:10191000D8340334A834AE342A34A8348D34513446
:10192000A83476347834A83467349F34A8346134CA
:10193000C634A8346534ED34A83471341434A93471
:1019400086343B34A934A5346234A934CC34893488
:10195000A934FC34B034A9343634D834A9347934B9
:10196000FF34A934C4342634AA3419344E34AA348A
:1019700077347534AA34DE349C34AA344E34C434FB
:10198000AA34C734EB34AA3449341334AB34D534D5
:101990003A34AB3469346234AB3407348A34AB3410
:1019A000AE34B134AB345E34D934AB341734013493
:1019B000AC34DA342834AC34A5345034AC347A3412
:1019C0007834AC345834A034AC343F34C834AC34FC
:1019D0003034F034AC3429341834AD342C34403441
:1019E000AD3438346834AD344E349034AD346C3466
:1019F000B834AD349434E034AD34C6340834AE3445
:101A000000343134AE3444345934AE3491348134FA
:101A1000AE34E734A934AE344734D234AE34B034C3
:101A2000FA34AE3423342334AF349F344B34AF34E0
:101A300024347434AF34B2349C34AF344A34C534B3
:101A4000AF34EB34ED34AF3496341634B0344A341A
:101A50003F34B03408346834B034CF349034B034C8
:101A60009F34B934B0347934E234B0345C340B345C
:101A7000B13448343434B1343F345D34B1343E345D
:101A80008634B1344734AF34B1345A34D834B134F5
:101A900076340134B2349B342A34B234CA345334E9
:101AA000B23403347D34B2344534A634B234913484
:101AB000CF34B234E634F834B23445342234B3345B
:101AC000AD344B34B3341F347534B3349A349E344C
:101AD000B3341F34C834B334AE34F134B334463481
:101AE0001B34B434E8344434B43493346E34B434F2
:101AF00048349834B4340734C234B434D034EB347A
:101B0000B434A2341534B5347D343F34B534633441
:101B10006934B53452349334B5344B34BD34B534B0
:101B20004D34E734B53459341134B6346F343B3462
:101B3000B6348F346534B634B8348F34B634EB34BD
:101B4000B934B6342834E434B6346F340E34B73490
:101B5000BF343834B73419346334B7347D348D34FA
:101B6000B734EB34B734B7346334E234B734E434E5
:101B70000C34B8346F343734B83405346234B83484
:101B8000A3348C34B8344C34B734B834FF34E13433
:101B9000B834BB340C34B93482343734B9345234A9
:101BA0006234B9342C348D34B9341034B834B93487
:101BB000FE34E234B934F6340D34BA34F8343834FF
:101BC000BA3404346434BA3419348F34BA343934FE
:101BD000BA34BA346334E534BA3496341034BB348E
:101BE000D4343B34BB341B346734BB346D3492344F
:101BF000BB34C934BD34BB342E34E934BB349E34D9
:101C00001434BC3418344034BC349B346B34BC348E
:101C100029349734BC34C134C234BC346334EE3418
:101C2000BC340F341A34BD34C5344534BD34863425
:101C30007134BD3450349D34BD342434C934BD3482
:101C40000334F534BD34EC342034BE34DF344C344A
:101C5000BE34DC347834BE34E334A434BE34F434DB
:101C6000D034BE341034FD34BE3436342934BF345D
:101C700066345534BF34A0348134BF34E434AD34D9
:101C8000BF343334DA34BF348C340634C034EF34E8
:101C90003234C0345D345F34C034D4348B34C03417
:101CA0005634B834C034E334E434C03479341134B5
:101CB000C1341A343E34C134C5346A34C1347B343F
:101CC0009734C1343B34C434C1340534F134C134A5
:101CD000D9341D34C234B8344A34C234A1347734D0
:101CE000C2349534A434C2349334D134C2349C34D5
:101CF000FE34C234AE342B34C334CC345834C33401
:101D0000F3348534C3342634B334C3346234E0341A
:101D1000C334A9340D34C434FB343A34C434573496
:101D20006834C434BD349534C4342E34C334C4341C
:101D3000AA34F034C43430341E34C534C0344B3487
:101D4000C5345B347934C5340134A734C534B13477
:101D5000D434C5346B340234C63431343034C634F0
:101D600001345E34C634DB348B34C634C034B93409
:101D7000C634B034E734C634AA341534C734AF346B
:101D80004334C734BE347134C734D9349F34C73474
:101D9000FD34CD34C7342D34FC34C73467342A3491
:101DA000C834AC345834C834FB348634C834563460
:101DB000B534C834BB34E334C8342A341234C9349B
:101DC000A5344034C9342A346F34C934BA349D340C
:101DD000C9345534CC34C934FA34FA34C934AA3449
:101DE0002934CA3465345834CA342B348734CA345D
:101DF000FC34B534CA34D734E434CA34BE34133472
:101E0000CB34AF344234CB34AB347134CB34B23412
:101E1000A034CB34C334CF34CB34E034FE34CB34B1
:101E200007342E34CC343A345D34CC3477348C34AB
:101E3000CC34BF34BB34CC341234EB34CC347034B7
:101E40001A34CD34DA344934CD344E347934CD3487
:101E5000CC34A834CD345634D834CD34EB340734B4
:101E6000CE348B343734CE3436346734CE34EC341D
:101E70009634CE34AD34C634CE347934F634CE34E0
:101E800050342634CF3432345634CF342034863470
:101E9000CF341834B634CF341B34E634CF342A343C
:101EA0001634D03443344634D03468347634D034A5
:101EB0009834A634D034D334D634D03419340734DB
:101EC000D1346A343734D134C7346734D1342E3402
:101ED0009834D134A134C834D1341F34F934D134D6
:101EE000A8342934D2343D345A34D234DC348A34E0
:101EF000D2348734BB34D2343D34EC34D234FF3462
:101F00001C34D334CC344D34D334A4347E34D33461
:101F10008734AF34D3347534E034D3346F34113470
:101F2000D43474344234D43485347334D434A13446
:101F3000A434D434C834D534D434FB340634D53442
:101F400038343834D53482346934D534D7349A347B
:101F5000D5343734CC34D534A234FD34D5341934A7
:101F60002F34D6349C346034D63429349234D63469
:101F7000C334C334D6346734F534D63418342734F4
:101F8000D734D3345834D7349B348A34D7346D346F
:101F9000BC34D7344C34EE34D73435342034D834D0
:101FA0002B345234D8342B348434D8343834B634C7
:101FB000D8345034E834D83473341A34D934A33490
:101FC0004C34D934DD347E34D9342434B134D9346A
:101FD0007634E334D934D3341534DA343C344834E9
:101FE000DA34B1347A34DA343234AD34DA34BE34FB
:101FF000DF34DA3456341234DB34FA344434DB342C
:084000000000050000000200B1
:02400E00623F0F
:1042000000000000000001000100010002000200A7
:10421000030003000300040004000400050005007F
:104220000600060006000700070007000800080057
:1042300008000900090009000A000A000A000A0033
:104240000B000B000B000C000C000C000C000C0011
:104250000D000D000D000D000E000E000E000E00F2
:104260000E000E000E000F000F000F000F000F00D9
:104270000F000F000F000F000F000F000F000F00C6
:104280000F000F000F000F000F000F000F000F00B6
:104290000F000F000F000F000F000F000E000E00A8
:1042A0000E000E000E000E000E000D000D000D00A1
:1042B0000D000C000C000C000C000C000B000B009F
:1042C0000B000A000A000A000A00090009000900A0
:1042D00008000800080007000700070006000600A5
:1042E00006000500050004000400040003000300AC
:1042F00003000200020001000100010000000000B4
:10430000000000000000FF00FF00FF00FE00FE00B4
:10431000FD00FD00FD00FC00FC00FC00FB00FB00BC
:10432000FA00FA00FA00F900F900F900F800F800C4
:10433000F800F700F700F700F600F600F600F600C8
:10434000F500F500F500F400F400F400F400F400CA
:10435000F300F300F300F300F200F200F200F200C9
:10436000F200F200F200F100F100F100F100F100C2
:10437000F100F100F100F100F100F100F100F100B5
:10438000F100F100F100F100F100F100F100F100A5
:10439000F100F100F100F100F100F100F200F20093
:1043A000F200F200F200F200F200F300F300F3007A
:1043B000F300F400F400F400F400F400F500F5005C
:1043C000F500F600F600F600F600F700F700F7003B
:1043D000F800F800F800F900F900F900FA00FA0016
:1043E000FA00FB00FB00FC00FC00FC00FD00FD00EF
:1043F000FD00FE00FE00FF00FF00FF0000000000C7
:00000001FF
